:020000040800F2
:1000000000800020E50C00082F0D0008650D000899
:1000100000000000000000000000000000000000E0
:10002000000000000000000000000000EB0C0008D1
:100030000000000000000000ED0C0008C1090008ED
:10004000EF0C0008F10C0008F30C0008F50C000898
:10005000F70C0008F90C0008FB0C0008FD0C000868
:10006000FF0C0008010D0008030D0008050D000835
:10007000070D0008090D00080B0D00080D0D000804
:100080000F0D0008110D0008130D0008150D0008D4
:10009000170D0008190D00081B0D00081D0D0008A4
:1000A0001F0D0008210D0008230D0008250D000874
:1000B000270D0008290D00082B0D00082D0D000844
:1000C0004543532E46573A30312E30302E303100D2
:1000D0000120C006014908607047C04608ED00E0F5
:1000E00010B51D4CA0688006400F411E032923D87F
:1000F0001A48C0467944097949008F442201171AE9
:10010000E16803220A40032A00D01548E168490645
:10011000490F491C00F02EFEE1684904490E48438E
:10012000E168490F491C00F025FE0AE07D2000022D
:1001300007E00120C00304E020688004410F084864
:10014000C84008490860A26892093C231340064A47
:10015000D258D040086010BD0010024000127A0052
:0C0160000024F400000000206C010008E6
:10016C000000000000000000000000000000000083
:10017C000000000000000000000000000000000073
:10018C000100000002000000030000000400000059
:10019C000600000007000000080000000900000035
:1001AC00D0B502AFFFB089B06E4600F031FA012035
:1001BC000104B160F061C0077060E648006830610E
:1001CC00E54800F021FB7F280FD080B2E34988423C
:1001DC0003D0E349884200D1FFE1DE480068316971
:1001EC00401ADD498842EBD9F7E100F0A1FDFD484A
:1001FC0000F00AFB0546401CF9D0A8B2D849884249
:10020C00DED0F84800F000FB0028F0D4E9B2C0B210
:10021C00022913D1FD2811D1FC488019F1694170D4
:10022C0079210170F04C62780F231340837022788F
:10023C000171C270052100F07DFBD8E7002923D1A4
:10024C00FF2821D1F14880197921817392224273C0
:10025C00822202737322C27263228272432242721E
:10026C00312202722122C271112282710223437146
:10027C00F36903710023C37082700B22427001700A
:10028C000F2100F057FBB2E7112912D1EE2810D143
:10029C0000F04EFD0024D94804710460052C17D0E1
:1002AC00D04800F0B1FA0028A1D4D4490855641CF8
:1002BC00F4E701292BD1FE2829D1D44880197921C2
:1002CC0001710022C2708270112242700170B1E77C
:1002DC00CA4CE078A1786278237853404B40434075
:1002EC00206800BA20602079834200D0C9E000F079
:1002FC001FFD0024022C46D0BA4800F085FA0028D5
:10030C0000D574E7C14989190855641CF2E74329E3
:10031C0023D1BC2821D100F00BFDB24800F074FAB7
:10032C00002800D563E70246093207218A43694653
:10033C00F16069468A1A95467061851C1446B26153
:10034C00002D4BD0A74800F05FFA002800D5A4E0A0
:10035C002070641C6D1EB269F2E7312933D1CE28AE
:10036C0031D100F0E5FC0024A44804710460052C94
:10037C0071D09C4800F048FA002800D537E79F4917
:10038C000855641CF3E7A14880194178FF244C40C0
:10039C000078A04275D1254608350720854300F02A
:1003AC00C7FC6846B0616846451BAD46641CEC2230
:1003BC002846214600F0EDFC2846214600F0BAFA0A
:1003CC00B069854613E700F0BDFC854800683169CB
:1003DC00401A8449884200D809E7FEE07169481C3C
:1003EC00C9B20346814D002B04D014786140521CD5
:1003FC005B1EF8E7B269105C814245D1E8680028C1
:10040C0003D57B4828607C4828600020B46871695B
:10041C0088423CDC115C06291BD3AA682242FCD121
:10042C00AA68AA603F22D200EB689343EB60C90034
:10043C00EA680A43EA60EA6802210A43EA60EA6869
:10044C002243EA60AA682242FCD1EA688A43EA6045
:10045C00B269401CDBE7694A1078517841409078CA
:10046C004840D1784140107981420AD100F060FCBB
:10047C005C4800F0C9F9002800D5B8E6411C8A0791
:10048C000ED000F05FFCB2E600F05CFC05E0E86822
:10049C0071680843E86000F04BFCF0688546A6E6FE
:1004AC007061B161F069010258488019FF22F16056
:1004BC0000F06FFC00254F4CB069A84209D04948A8
:1004CC0000F0A2F9002804D45049891948556D1C34
:1004DC00F2E7216804204907014600D51421605039
:1004EC007469A54200DC82E63E4800F08DF90028D4
:1004FC0000D57CE600212246A14205DC434B9B192A
:10050C005B5C5A40491CF7E7D1B28142B9D13B49F7
:10051C00086800BA08603A49884200D265E60019BA
:10052C003849884200D960E6F01D1930F16800F0B6
:10053C002FFC00242D4D7069844213DC3348801944
:10054C000019F11D19310A192F4900F03BFA10342A
:10055C00F1E7C0461000002088130000FFFF0000E8
:10056C00FEFF0000E868002803D5214828602248D7
:10057C002860B069C010F0600021B468F068814256
:10058C0022DAAA682242FCD1AA68AA60B161CA0028
:10059C00F31D19339C18606870619B5817480568E7
:1005AC001248C068F4692043B4681049C860AB5065
:1005BC00A8180E4DBFF36F8F71694160A868204277
:1005CC00FCD1B169491CD9E7E868F1698843E86056
:1005DC00E86871680843E86007E600F05FF9ECE54D
:1005EC001000002088130000005801400820024031
:1005FC0023016745140C0050AB89EFCD040000209B
:10060C0000300008FFEF0108B40E000820010000C4
:10061C00F0B583B06E4800687D21C90000F0A4FBE2
:10062C00401E010E0DD16B496B4A50606B4803683C
:10063C000B400321890759180160002090600720A6
:10064C0010600120054604020020C343644E30684C
:10065C00C00506D42046F43019461F4600F07AF93E
:10066C003B4602945F490F46BF3730683842FAD098
:10067C002C045D488169C9B2AA2903D08169C9B229
:10068C00CC2927D1C168002903D5584901605849A4
:10069C000160C168490003D5564941605649416023
:1006AC008169FF22914381618169EC220A43826155
:1006BC0081682142FCD16904C2680A43C260816826
:1006CC002142FCD1E906C2680A43C2606420194683
:1006DC0000F040F9706B0B2101437163CF20810452
:1006EC000526300702688A4302604521C904026866
:1006FC000A43026003210905C2688A43C26001955E
:10070C002905C2680A43C2600F221102436A8B4357
:10071C004362416A029B19434162416AF023994347
:10072C004162436A10210B4343621204436A9343B0
:10073C004362426A22434262304D28683022904321
:10074C0028602868C02290432860286808432860E5
:10075C002868402101432960019CA103204A106CA8
:10076C000843106426480268A2430260220703680B
:10077C00934303602203036813430360E20303689B
:10078C009343036002683A432746026002680C23D5
:10079C001343036002681B4B1343036082680A43D4
:1007AC0082601049C160016821430160002E0CD0A9
:1007BC000420A8619624204600F0EEF8B804A86145
:1007CC00204600F0E9F8761EF0E703B0F0BDC04615
:1007DC0000000020FFFFFF0010E000E020ED00E033
:1007EC00001002404103000008200240230167452D
:1007FC00AB89EFCD3B2A19087F6E5D4C000C005085
:08080C00003801400000FF0369
:10081400F0B581B01F4A146813681F49204D0E6853
:10082400B60610D41668F61A86420CD21668361B21
:100834004B2EF4D314682F6804267F07374600D55F
:1008440014277E51EBE71268D21A82420FD2134862
:100854000A6812070FD40A68520712D40A6892076A
:1008640011D40A68D20710D18868C0B20FE0002002
:10087400C043401E0BE008224A608968C9B2009157
:1008840005E0042202E0022200E001224A6000B2F4
:1008940001B0F0BD100000201C380140FFFF000033
:0408A400140C0050E0
:1008A800F0B581B0012002031A490B6813430B60AD
:1008B800194B9C6804439C6000241848184D1D4E31
:1008C800AC4205D227583FBA1F602418A419F7E78D
:1008D800144C24681B68A34215D10B6893430B6022
:1008E800124900248C604C600C6072B61049086094
:1008F800016881F3088862B640688047E1437D203B
:1009080000F02AF8FAE7FA20074900F025F801B0C4
:10091800F0BDC046381002400030024000300008E8
:10092800FCBF0100FCEF01088813000010E000E0A4
:0809380008ED00E004D0FFF718
:1009400010B50022054B8A4206DA1C682406FCD545
:10095000845CDC60521CF6E710BDC0461C380140C8
:10096000F0B581B0009105460126B0040B4F386008
:100970000B4804680A480068001B009988420AD2A4
:1009800008203860284600F00DF8F004386028464A
:1009900000F008F8EEE701B0F0BDC046180C0050BA
:0409A0001000002023
:1009A40081B005490A6800920A68009BD21A824203
:0C09B400FAD301B07047C04610000020CC
:1009C00002480168491C01607047C04610000020C1
:1009D000F0B591B00023102B03D0C45CD4545B1C41
:1009E000F9E78D4801608D48026000228C48102A8A
:1009F0000BD08B5C835483188C1865785D70A57858
:100A00009D70E478DC70121DF1E70421844C2C29E0
:100A100048D08D000C22102A06D0A35C10AEB61868
:100A20000C3E3370521CF6E710AEF778B37872784C
:100A30003678880703D00F970E93134612E0794853
:100A40000D910146865D10A80F96C670CE5D0E967C
:100A50008670CB5C43708A5C0D998E08724FBE5DC8
:100A6000564006706E4F7A19104610380078704064
:100A700078550120284316460F3E36785E403E5496
:100A80000220284313460E3B1B780E9E73403B54B6
:100A9000032028430D3A12780F9B5A403A54241DE4
:100AA000491CB4E70A2000F0C1F8092400F0DAF884
:100AB00000F0F6F8200600D1A9E00194E0B200F0C1
:100AC000B5F85648006807900020102800D19BE038
:100AD000079A11180F9001200B5602200D560C4654
:100AE00005912E465E400F981056C10902460390AC
:100AF0001B200140570079400A464E4004910321D3
:100B000061560E914E40D90901405C000A94614043
:100B10000B914E4054007AB2D109014061404E40E1
:100B2000069162B2D2090240490051400C914E40F8
:100B3000E90901406C0061400D914A00089264B2DD
:100B4000E109014051404E400F4602910B994A0085
:100B500054B2E10901400A9C64B2E40904405440E3
:100B60000A9462004A4009925640089949B2C9095C
:100B700001407A004A40089256400E99CA09024044
:100B800049004A40540067B2FF09074049B2C90909
:100B9000014061404800784046400F9C079F3E5509
:100BA0002E46039F7E400E9C66400B9C66400D9C2B
:100BB00066400A9C66400C9C6640099C66404E401C
:100BC000089C66404640059C66707B4053400C9AEA
:100BD00053405D40049A55400A9A5540099E75401D
:100BE0004D40089F7D404540E5700E9A5340069A5F
:100BF00053400D9A5340029A534073407B40434008
:100C00000F98A370001D60E7019C641E4EE7002052
:100C100000F00CF811B0F0BD140000200C00002012
:0C0C200018000020C40E0008B00D0008F1
:100C2C00B0B500010A4908180A4909680022042ACB
:100C3C000CD00023042B05D0C45CCD5C6540CD5496
:100C4C005B1CF7E7091D001D521CF0E7B0BDC04648
:080C5C00180000200C0000202C
:100C64000D480068417B427A42734279437843716C
:100C7400427241708178827A827081728179827B3A
:100C840082718173C178C279C270C27AC271C27B27
:0C0C9400C173C2727047C0460C00002003
:100CA00010B5094800680021084A04290AD0002329
:100CB000102B04D0C45C145DC4541B1DF8E7401C09
:100CC000491CF2E710BDC0460C000020C40F00080C
:100CD000034C206804348047FBE7FFF767FAFEE720
:040CE000C410000834
:060CE400FFF7F4F9F2E74E
:020CEA00FEE723
:020CEC00FEE721
:020CEE00FEE71F
:020CF000FEE71D
:020CF200FEE71B
:020CF400FEE719
:020CF600FEE717
:020CF800FEE715
:020CFA00FEE713
:020CFC00FEE711
:020CFE00FEE70F
:020D0000FEE70C
:020D0200FEE70A
:020D0400FEE708
:020D0600FEE706
:020D0800FEE704
:020D0A00FEE702
:020D0C00FEE700
:020D0E00FEE7FE
:020D1000FEE7FC
:020D1200FEE7FA
:020D1400FEE7F8
:020D1600FEE7F6
:020D1800FEE7F4
:020D1A00FEE7F2
:020D1C00FEE7F0
:020D1E00FEE7EE
:020D2000FEE7EC
:020D2200FEE7EA
:020D2400FEE7E8
:020D2600FEE7E6
:020D2800FEE7E4
:020D2A00FEE7E2
:020D2C00FEE7E0
:0E0D2E0080B50020C143FA20FFF713FE80BD00
:100D3C0080B582B001A8792101700121FFF7FAFD7D
:040D4C0002B080BDB4
:100D500080B582B001A81F2101700121FFF7F0FDCD
:040D600002B080BDA0
:100D640080B57D2080000021C943FFF7F7FD80BDD9
:100D74000A000FD00300400800E052008242FCD970
:100D8400002000E05208934200D39B1A40418A425B
:080D9400F8D170470020704700
:100D9C0000220B0011001A00002A02D0013A8154E3
:040DAC00FCD17047BF
:100DB0008D01020408102040801B366CD8AB4D9A80
:100DC0002F5EBC63C697356AD4B37DFAEFC59139FF
:100DD00072E4D3BD61C29F254A943366CC831D3A29
:100DE00074E8CB8D01020408102040801B366CD8BB
:100DF000AB4D9A2F5EBC63C697356AD4B37DFAEFCC
:100E0000C5913972E4D3BD61C29F254A943366CC43
:100E1000831D3A74E8CB8D01020408102040801B2A
:100E2000366CD8AB4D9A2F5EBC63C697356AD4B387
:100E30007DFAEFC5913972E4D3BD61C29F254A9412
:100E40003366CC831D3A74E8CB8D01020408102070
:100E500040801B366CD8AB4D9A2F5EBC63C697356D
:100E60006AD4B37DFAEFC5913972E4D3BD61C29FF4
:100E7000254A943366CC831D3A74E8CB8D01020475
:100E800008102040801B366CD8AB4D9A2F5EBC6397
:100E9000C697356AD4B37DFAEFC5913972E4D3BDF4
:0F0EA00061C29F254A943366CC831D3A74E8CB18
:040EB000E100000855
:100EB4005C383657603D0E38611E4E216219476218
:100EC400637C777BF26B6FC53001672BFED7AB7603
:100ED400CA82C97DFA5947F0ADD4A2AF9CA472C0AE
:100EE400B7FD9326363FF7CC34A5E5F171D831151B
:100EF40004C723C31896059A071280E2EB27B2753C
:100F040009832C1A1B6E5AA0523BD6B329E32F84B3
:100F140053D100ED20FCB15B6ACBBE394A4C58CFAB
:100F2400D0EFAAFB434D338545F9027F503C9FA87F
:100F340051A3408F929D38F5BCB6DA2110FFF3D24D
:100F4400CD0C13EC5F974417C4A77E3D645D197301
:100F540060814FDC222A908846EEB814DE5E0BDBFB
:100F6400E0323A0A4906245CC2D3AC629195E47932
:100F7400E7C8376D8DD54EA96C56F4EA657AAE088C
:100F8400BA78252E1CA6B4C6E8DD741F4BBD8B8A27
:100F9400703EB5664803F60E613557B986C11D9E8D
:100FA400E1F8981169D98E949B1E87E9CE5528DF04
:100FB4008CA1890DBFE6426841992D0FB054BB1630
:100FC40052096AD53036A538BF40A39E81F3D7FBBA
:100FD4007CE339829B2FFF87348E4344C4DEE9CB04
:100FE400547B9432A6C2233DEE4C950B42FAC34E79
:100FF400082EA16628D924B2765BA2496D8BD1252F
:1010040072F8F66486689816D4A45CCC5D65B692D2
:101014006C704850FDEDB9DA5E154657A78D9D8476
:1010240090D8AB008CBCD30AF7E45805B8B3450696
:10103400D02C1E8FCA3F0F02C1AFBD0301138A6BB0
:101044003A9111414F67DCEA97F2CFCEF0B4E673E0
:1010540096AC7422E7AD3585E2F937E81C75DF6E8E
:1010640047F11A711D29C5896FB7620EAA18BE1BF4
:10107400FC563E4BC6D279209ADBC0FE78CD5AF49A
:101084001FDDA8338807C731B11210592780EC5FE0
:1010940060517FA919B54A0D2DE57A9F93C99CEF3C
:1010A400A0E03B4DAE2AF5B0C8EBBB3C835399613D
:1010B400172B047EBA77D626E169146355210C7D7B
:1010C400F51000080400002005000000F5100008D9
:1010D4000C000020BC0000000711000800000020E4
:0C10E400F010000804000000DB0C000805
:0410F0000024F400E4
:1010F400206861680834002200E042540139FCD5BC
:02110400704732
:1011060020686168A2680C3401E08B5C8354013A64
:04111600FBD570474E
:0400000508000CE5FE
:00000001FF
